BL51 BANKED LINKER/LOCATER V6.22.2.0                                                    03/16/2023  09:43:04  PAGE 1


BL51 BANKED LINKER/LOCATER V6.22.2.0, INVOKED BY:
C:\KEIL_V5\C51\BIN\BL51.EXE .\Release\system_FE81001.obj, .\Release\STARTUP.obj, .\Release\main.obj TO .\Release\Sample_
>> DrvUART_Int_RX REGFILE (.\Release\Sample_DrvUART_Int_RX.ORC) PRINT (.\Sample_DrvUART_Int_RX.m51) RAMSIZE (256) CODE (
>> 0X0000-0X1FFF) XDATA (0X8000-0X87FF)


MEMORY MODEL: SMALL


INPUT MODULES INCLUDED:
  .\Release\system_FE81001.obj (SYSTEM_FE81001)
  .\Release\STARTUP.obj (?C_STARTUP)
  .\Release\main.obj (MAIN)
  C:\KEIL_V5\C51\LIB\C51S.LIB (?C_INIT)
  C:\KEIL_V5\C51\LIB\C51S.LIB (?C_IBP)


LINK MAP OF MODULE:  .\Release\Sample_DrvUART_Int_RX (SYSTEM_FE81001)


            TYPE    BASE      LENGTH    RELOCATION   SEGMENT NAME
            -----------------------------------------------------

            * * * * * * *   D A T A   M E M O R Y   * * * * * * *
            REG     0000H     0008H     ABSOLUTE     "REG BANK 0"
            DATA    0008H     000BH     UNIT         ?DT?MAIN
            DATA    0013H     0006H     UNIT         ?DT?_DELAY?MAIN
            DATA    0019H     0001H     UNIT         ?DT?UARTISR?MAIN
            DATA    001AH     0001H     UNIT         ?C?LIB_DATA
                    001BH     0005H                  *** GAP ***
            BIT     0020H.0   0000H.1   UNIT         ?BI?MAIN
                    0020H.1   0000H.7                *** GAP ***
            IDATA   0021H     0001H     UNIT         ?STACK

            * * * * * * *   C O D E   M E M O R Y   * * * * * * *
            CODE    0000H     0003H     ABSOLUTE     
            CODE    0003H     003BH     UNIT         ?PR?_DELAY?MAIN
            CODE    003EH     0023H     UNIT         ?PR?UART_CONFIG?MAIN
            CODE    0061H     0001H     UNIT         ?PR?SYSTEMINIT?SYSTEM_FE81001
                    0062H     0001H                  *** GAP ***
            CODE    0063H     0003H     ABSOLUTE     
            CODE    0066H     009DH     UNIT         ?C_C51STARTUP
            CODE    0103H     0090H     UNIT         ?PR?IOCONFIG?MAIN
            CODE    0193H     0061H     UNIT         ?PR?UARTISR?MAIN
            CODE    01F4H     0027H     UNIT         ?PR?MAIN?MAIN
            CODE    021BH     0022H     UNIT         ?PR?TX_MODE?MAIN
            CODE    023DH     0019H     UNIT         ?PR?RX_MODE?MAIN
            CODE    0256H     0017H     UNIT         ?PR?CLKCONFIG?MAIN
            CODE    026DH     0012H     UNIT         ?C_INITSEG



OVERLAY MAP OF MODULE:   .\Release\Sample_DrvUART_Int_RX (SYSTEM_FE81001)


SEGMENT
  +--> CALLED SEGMENT
---------------------
BL51 BANKED LINKER/LOCATER V6.22.2.0                                                  03/16/2023  09:43:04  PAGE 2


?C_C51STARTUP
  +--> ?PR?MAIN?MAIN
  +--> ?C_INITSEG

?PR?MAIN?MAIN
  +--> ?PR?UART_CONFIG?MAIN
  +--> ?PR?RX_MODE?MAIN
  +--> ?PR?_DELAY?MAIN

?PR?UART_CONFIG?MAIN
  +--> ?PR?CLKCONFIG?MAIN
  +--> ?PR?IOCONFIG?MAIN

*** NEW ROOT ***************************************************

?PR?UARTISR?MAIN
  +--> ?PR?TX_MODE?MAIN



SYMBOL TABLE OF MODULE:  .\Release\Sample_DrvUART_Int_RX (SYSTEM_FE81001)

  VALUE           TYPE          NAME
  ----------------------------------

  -------         MODULE        SYSTEM_FE81001
  C:0000H         SYMBOL        _ICE_DUMMY_
  C:0061H         PUBLIC        SystemInit
  -------         PROC          SYSTEMINIT
  C:0061H         LINE#         38
  C:0061H         LINE#         39
  C:0061H         LINE#         41
  -------         ENDPROC       SYSTEMINIT
  -------         ENDMOD        SYSTEM_FE81001

  -------         MODULE        ?C_STARTUP
  C:0066H         SEGMENT       ?C_C51STARTUP
  I:0021H         SEGMENT       ?STACK
  C:0000H         PUBLIC        ?C_STARTUP
  D:00E0H         SYMBOL        ACC
  D:00F0H         SYMBOL        B
  D:0083H         SYMBOL        DPH
  D:0082H         SYMBOL        DPL
  N:0001H         SYMBOL        IBPSTACK
  N:0100H         SYMBOL        IBPSTACKTOP
  N:0080H         SYMBOL        IDATALEN
  C:0069H         SYMBOL        IDATALOOP
  N:0000H         SYMBOL        PBPSTACK
  N:0100H         SYMBOL        PBPSTACKTOP
  N:0000H         SYMBOL        PDATALEN
  N:0000H         SYMBOL        PDATASTART
  N:0000H         SYMBOL        PPAGE
  N:0000H         SYMBOL        PPAGEENABLE
  D:00A0H         SYMBOL        PPAGE_SFR
  D:0081H         SYMBOL        SP
  C:0066H         SYMBOL        STARTUP1
  N:0000H         SYMBOL        XBPSTACK
BL51 BANKED LINKER/LOCATER V6.22.2.0                                                  03/16/2023  09:43:04  PAGE 3


  N:0000H         SYMBOL        XBPSTACKTOP
  N:0800H         SYMBOL        XDATALEN
  C:0074H         SYMBOL        XDATALOOP
  N:8000H         SYMBOL        XDATASTART
  C:0000H         LINE#         126
  C:0066H         LINE#         133
  C:0068H         LINE#         134
  C:0069H         LINE#         135
  C:006AH         LINE#         136
  C:006CH         LINE#         140
  C:006FH         LINE#         141
  C:0071H         LINE#         145
  C:0073H         LINE#         147
  C:0074H         LINE#         148
  C:0075H         LINE#         149
  C:0076H         LINE#         150
  C:0078H         LINE#         151
  C:007AH         LINE#         170
  C:007DH         LINE#         185
  C:0080H         LINE#         196
  -------         ENDMOD        ?C_STARTUP

  -------         MODULE        MAIN
  C:0000H         SYMBOL        _ICE_DUMMY_
  D:0090H         PUBLIC        P1
  D:00B0H         PUBLIC        P3
  D:0008H         SYMBOL        rx_buf
  D:00A8H         PUBLIC        IE
  C:0003H         PUBLIC        _delay
  C:003EH         PUBLIC        UART_config
  D:00B8H         PUBLIC        IP
  C:01F4H         PUBLIC        main
  C:0193H         PUBLIC        UARTISR
  D:0098H         PUBLIC        SCON
  C:0256H         PUBLIC        CLKConfig
  D:0088H         PUBLIC        TCON
  B:0020H.0       PUBLIC        Rx_OK
  D:0012H         SYMBOL        cnt
  C:023DH         PUBLIC        Rx_mode
  C:021BH         PUBLIC        Tx_mode
  D:00C8H         PUBLIC        T2CON
  C:0103H         PUBLIC        IOConfig
  D:00D0H         PUBLIC        PSW
  -------         PROC          _DELAY
  D:0013H         SYMBOL        cnt
  -------         DO            
  D:0015H         SYMBOL        i
  D:0017H         SYMBOL        j
  -------         ENDDO         
  C:0003H         LINE#         37
  C:0007H         LINE#         38
  C:0007H         LINE#         41
  C:0018H         LINE#         42
  C:003DH         LINE#         44
  -------         ENDPROC       _DELAY
  -------         PROC          UARTISR
  -------         DO            
BL51 BANKED LINKER/LOCATER V6.22.2.0                                                  03/16/2023  09:43:04  PAGE 4


  D:0019H         SYMBOL        int_stat
  -------         ENDDO         
  C:0193H         LINE#         56
  C:01B0H         LINE#         58
  C:01B7H         LINE#         60
  C:01C4H         LINE#         62
  C:01CBH         LINE#         64
  C:01D0H         LINE#         66
  C:01D3H         LINE#         68
  C:01D9H         LINE#         71
  -------         ENDPROC       UARTISR
  -------         PROC          RX_MODE
  C:023DH         LINE#         83
  C:023DH         LINE#         84
  C:023DH         LINE#         86
  C:0243H         LINE#         89
  C:0249H         LINE#         92
  C:024FH         LINE#         93
  C:0255H         LINE#         94
  -------         ENDPROC       RX_MODE
  -------         PROC          TX_MODE
  C:021BH         LINE#         97
  C:021BH         LINE#         98
  C:021BH         LINE#         101
  C:0221H         LINE#         104
  C:0227H         LINE#         107
  C:022DH         LINE#         108
  C:023CH         LINE#         109
  -------         ENDPROC       TX_MODE
  -------         PROC          IOCONFIG
  C:0103H         LINE#         121
  C:0103H         LINE#         122
  C:0103H         LINE#         125
  C:0119H         LINE#         126
  C:012FH         LINE#         129
  C:0150H         LINE#         130
  C:0171H         LINE#         133
  C:0192H         LINE#         135
  -------         ENDPROC       IOCONFIG
  -------         PROC          CLKCONFIG
  C:0256H         LINE#         147
  C:0256H         LINE#         148
  C:0256H         LINE#         150
  C:0261H         LINE#         153
  C:026CH         LINE#         154
  -------         ENDPROC       CLKCONFIG
  -------         PROC          UART_CONFIG
  C:003EH         LINE#         156
  C:003EH         LINE#         157
  C:003EH         LINE#         158
  C:0041H         LINE#         159
  C:0044H         LINE#         161
  C:0060H         LINE#         163
  -------         ENDPROC       UART_CONFIG
  -------         PROC          MAIN
  C:01F4H         LINE#         175
  C:01F4H         LINE#         176
BL51 BANKED LINKER/LOCATER V6.22.2.0                                                  03/16/2023  09:43:04  PAGE 5


  C:01F4H         LINE#         177
  C:01F7H         LINE#         178
  C:01FAH         LINE#         180
  C:01FFH         LINE#         181
  C:0204H         LINE#         183
  C:0204H         LINE#         184
  C:0204H         LINE#         185
  C:0211H         LINE#         186
  C:0218H         LINE#         188
  -------         ENDPROC       MAIN
  -------         ENDMOD        MAIN

  -------         MODULE        ?C_IBP
  D:001AH         PUBLIC        ?C_IBP
  -------         ENDMOD        ?C_IBP



FUNCTION REGISTER MASKS


FUNCTION . . . . . REG MASK
---------------------------

CLKCONFIG. . . . . @0xe301
IOCONFIG . . . . . @0xe301
MAIN . . . . . . . @0xf303
RX_MODE. . . . . . @0xa300
SYSTEMINIT . . . . @0x8000
TX_MODE. . . . . . @0xe303
UART_CONFIG. . . . @0xe301
_DELAY . . . . . . @0xf000

*** WARNING L16: UNCALLED SEGMENT, IGNORED FOR OVERLAY PROCESS
    SEGMENT: ?PR?SYSTEMINIT?SYSTEM_FE81001

Program Size: data=28.1 xdata=0 code=638
LINK/LOCATE RUN COMPLETE.  1 WARNING(S),  0 ERROR(S)
